:020000040000FA
:040000008A112D280C
:08000800FE00030E8301A300BA
:100010000A08A4008A01262882070D340E341334FE
:100020001534163419341A341C3423342534263448
:1000300029342A342C343234343482072A342A3492
:100040002A342A342A342A3438342C347F08A6003F
:100050000408A7002008A200792983169F018312B3
:100060009F019A019C0183160510851005118515C5
:1000700005163730950081138312BF01C001C101FD
:10008000C201C3104311F729D5005308D800D50683
:10009000550EF039D800D5065508D600D7015608B8
:1000A000D900D8015408DA00DB015A085804DC00F2
:1000B0005B085904DD000310570CDF00560CDE000E
:1000C0000330A0000310DF0CDE0CA00B62285E08DA
:1000D0005C06E0005F085D06E1000310560DE200DB
:1000E000570DE3000310E20DE30D0310E20DE30DE5
:1000F00062086006E40063086106E5006408A00089
:100100006508A1000800C800FC3092058730920500
:100110004808831692008312121583168C140B174D
:100120008B170800C6007D107D08850046088328CF
:10013000C001C101C2014315C31408007D107D0830
:100140008500C31008002010C31820140800C3182D
:10015000A7280800C900CB01FF30CC00CD00033038
:100160004907D100033049020319BA28031CBA28F1
:1001700020100800A72083124C08D3004D08D4009B
:100180005108442083122008CC002108CD00510ED4
:100190000F39CE0033304B078400831300308A00C0
:1001A0004E080C2080008312CB0A0F305105CE0080
:1001B00033304B078400831300308A004E080C2034
:1001C00080008312CB0A4908D200CA0121294C08B9
:1001D000D3004D08D40046084A078400831347180B
:1001E00083170008442083122008CC002108CD008A
:1001F00046084A078400831347188317000E0F39F7
:10020000CE0033304B078400831300308A004E0841
:100210000C2080008312CB0A46084A07840083130F
:10022000471883170F300005CE0033304B0784008A
:10023000831300308A004E080C2080008312CB0A02
:10024000CA0A4A085202031DE728CC09CD09031047
:100250004D0CCF004C0CCE000330A0000310CF0C8F
:10026000CE0CA00B2E290F304E05D00033304B079B
:100270008400831300308A0050080C208000831211
:10028000CB0A0F304C05CE0033304B07840083136C
:1002900000308A004E080C2080008312CB0A4D0EDD
:1002A0000F39CE00CF010F304E05D00033304B0751
:1002B0008400831300308A0050080C2080008312D1
:1002C000CB0A4D08CE00CF010F304E05D0003330A1
:1002D0004B078400831300308A0050080C208000F4
:1002E0008312CB0A08304B07BF00982083122014DA
:1002F00008008C1CEA298C1042082A14031D2A10BD
:10030000AA14C3182A1CAA10AA1CE129431DB62945
:100310004108FF000130A8007F0891290310A80DB3
:10032000FF03031D8E2900308A0040081D20831220
:10033000A00028082005A90029080319A1297D1477
:10034000A2297D107D088500C10A063041020319EB
:10035000AB29031CAD29C101C00A083040020319B2
:10036000B329031CE1294311C001E12940083F02E0
:100370000319BC290318BE299E20E1294108FF006A
:100380000130A8007F08C7290310A80DFF03031D33
:10039000C429333040078400831328080005A900CE
:1003A00029080319D5297D14D6297D107D088500DB
:1003B000C10A063041020319DF29031CE129C101EA
:1003C000C00A8312C20A073042020319EA29031C39
:1003D000EA29C2012208A000270884002608FF009D
:1003E00024088A00230E8300FE0E7E0E0900FA30D8
:1003F0009220FD107D08831285007D117D08850007
:10040000AE01AF010130B200B001B101431483125B
:1004100003139330A0001A30A1000A128A11A10B15
:100420000D2A0A128A11A00B0B2A000000000000FE
:1004300000000000051A342A831203139C30A00028
:100440007F30A1000A128A11A10B222A0A128A11F6
:10045000A00B202A0000431C342A4310051A342A1A
:100460003230AF000330B000051A43143008C31611
:100470000319C31231084317031D4313C317C31ACB
:10048000431FC3134414C31B851D4410441C702A0E
:10049000A3208312C4102018C414C418702A013079
:1004A000AB000130AC003208AD002B30C600C701F4
:1004B0000330AA208312C4112018C415C41D702A49
:1004C0000F30B100B0033008031D6E2A64303202D1
:1004D000031D6D2A0130B2006E2AB20A6430AE00EC
:1004E0002E08031D772A7D117D0885007B2A7D1546
:1004F0007D088500AE032F08031D822AFD107D08AC
:100500008500862AFD147D088500AF03A320831291
:100510004510201845144518C510451CC514310850
:10052000451503194511C515C518451DC511C51D2E
:06053000072AB103072AAF
:02400E00C43FAD
:00000001FF
